:100000000C948F050C94D3050C94D3050C94D30554
:100010000C94D3050C94D3050C94D3050C94D30500
:100020000C94D3050C94D3050C94F9190C94CB1AA9
:100030000C942D280C94D3050C94D3050C94D30563
:100040000C94D3050C9486060C94D3050C94D3051C
:100050000C94D3050C9495280C94D3050C94D305DB
:100060000C94D3050C94D3050C94D3050C94D305B0
:100070000C94D3050C94D3050C94D3050C94D305A0
:100080000C94DB0F0C94D3050C94D3050C94D3057E
:100090000C94D3050C94D3050C94D3050C94D30580
:1000A0000C94D3050C94D3050C94D305EE060007ED
:1000B000140726072E074407920792079207920714
:1000C0009207920752078107381B5A1B481C5A1B7C
:1000D000481C9F1BC21B481C171C2A1C141F141FE2
:1000E000431F431F821FA21FF820F820AD1FF820D6
:1000F0005D205D20C420CD20F820F2206A206A20F7
:100100006A206A206A206A206A206A206A206A209F
:100110006A206A206A206A206A206A207A20882061
:100120008F209620A02007634236B79BD8A71A39A4
:10013000685618AEBAAB558C1D3CB7CC5763BD6D35
:10014000EDFD753EF6177231BF000000803F0800DC
:100150000000BE922449123EABAAAA2ABECDCCCC46
:100160004C3E00000080BEABAAAAAA3E00000000E0
:10017000BF000000803F0000000000084178D3BBB2
:100180004387D1133D190E3CC3BD4282AD2B3E685F
:10019000EC8276BED98FE1A93E4C80EFFFBE01C450
:1001A000FF7F3F0000000000000000000000000092
:1001B000000000010204060A0F17202C3A4A5D7164
:1001C000879DB3C7DAE9F5FCFFFCF5E9DAC7B39D13
:1001D00087715D4A3A2C20170F0A060402010000BD
:1001E00000000000000000002B0014001A000800AE
:1001F000150017001C0018000C00120013002A0044
:10020000290004001600070009000A000B000D0079
:100210000E000F0033003400E1001D001B0006003B
:1002200019000500110010003600370038002800C2
:100230000530E000E200E30003302C002C00043025
:100240005000510052004F002B0014001A0009000A
:1002500013000A000D000F0018001C0033002A00D4
:100260002900040015001600170007000B001100FC
:1002700008000C0012003400E1001D001B00060005
:10028000190005000E001000360037003800280065
:100290001450E000E200E30003302C002C00043096
:1002A0005000510052004F002B0034003600370040
:1002B00013001C0009000A00060015000F002A00A8
:1002C000290004001200080018000C0007000B00B1
:1002D0001700110016003800E100330014000D0073
:1002E0000E001B00050010001A0019001D00280058
:1002F0000530E000E200E30003302C002C00043065
:100300005000510052004F0035021E021F02200211
:1003100021022202230224022502260227022A00A9
:100320004C003A003B003C003D003E003F002D02E7
:100330002E022F0230023102010040004100420033
:100340004300440045003202640201000100010044
:100350000100010001000100010001000100010095
:10036000AB00AA00A900AE0035001E001F0020004F
:1003700021002200230024002500260027002A0057
:100380004C003A003B003C003D003E003F002D0089
:100390002E002F00300031000100400041004200DB
:1003A000430044004500320032000100010001001A
:1003B0000100010001000100010001000100010035
:1003C000AB00AA00A900AE001E001E001E001E0009
:1003D0001E001E001E001E001E001E001E001E002D
:1003E000000014001A000800150017001C00180077
:1003F0000C00120013002F0000000400160007007C
:1004000009000A000B000D000E000F00330034003D
:100410000D3000000000060019000000000011006F
:1004200010000000000000000000000000000000BC
:1004300000000000000000000000000000000000BC
:1004400000000000000000000000000000000000AC
:10045000000000000000000000000000000000009C
:10046000000000000000000000000000000000008C
:1007E00000000000000000000100005001000100B6
:1007F00001000100010001000100010001004C00A6
:10080000010001000100205021501350125000300F
:10081000013002300C3001000100275026502350D7
:10082000245028502950010001000100010001005E
:1008300001000100010001000100010001000100B0
:1008400001000100010001000000000000000000A4
:100850002A2B28000000000000000000000000001B
:1008600000000029000000002C1E34202122243426
:100870002627252E362D3738271E1F2021222324F8
:1008800025263333362E37381F0405060708090A94
:100890000B0C0D0E0F101112131415161718191A30
:1008A0001B1C1D2F3130232D350405060708090AAE
:1008B0000B0C0D0E0F101112131415161718191A10
:1008C0001B1C1D2F3130354C0000000000000000C3
:1008D0000000000000000000000000000000000018
:1008E0000000000000000000000101010101010002
:1008F00001010101000000000000000000000000F4
:1009000000000100010001010101010101010101DB
:1009100001010101010101010101010101010101C7
:1009200001010100000001010000000000000000C2
:1009300000000000000000000000000000000000B7
:100940000000000101010100280354006800650057
:10095000200050006C0061006E0063006B002000FE
:100960004B006500790062006F0061007200640056
:1009700000002C034F007200740068006F006C00D0
:1009800069006E0065006100720020004B00650088
:10099000790062006F006100720064007300000063
:1009A0000403090409026D00040100A0FA0904000F
:1009B000000103010100092111010001223F00078C
:1009C00005810308000A090401000103010200096E
:1009D0002111010001224D000705820308000A09C8
:1009E0000402000103000000092111010001223668
:1009F000000705830308000A09040300010300003F
:100A000000092111010001223900070584031000AB
:100A1000011201100100000008EDFE6060010001FC
:100A200002000105010906A101050719E029E715E2
:100A30000025019508750181020508190129059510
:100A400005750191029501750391010507190029AA
:100A50007715002501957875018102C0050109808F
:100A6000A101850216010026B7001A01002AB7006D
:100A7000751095018100C0050C0901A101850316BF
:100A80000100269C021A01002A9C02751095018122
:100A900000C005010902A1010901A1000509190110
:100AA000290515002501950575018102950175033C
:100AB00081010501093009311581257F95027508ED
:100AC000810609381581257F950175088106050C79
:100AD0000A38021581257F950175088106C0C00579
:100AE000010906A101050719E029E715002501956F
:100AF0000875018102950175088101050819012910
:100B00000595057501910295017503910105071978
:100B10000029FF150025FF950675088100C01124E6
:100B20001FBECFEFDAE0DEBFCDBF04B603FE24C0A8
:100B300080915E0490915F04A0916004B091610483
:100B40008730904BA740B04BB9F410925E041092DE
:100B50005F04109260041092610414BE84B7877F12
:100B600084BF88E10FB6F894809360001092600013
:100B70000FBEE0E0F8E3099513E0A0E0B1E0EEEB92
:100B8000F4E602C005900D92A030B107D9F714E049
:100B9000A0E0B3E001C01D92AE35B107E1F70E94BD
:100BA0003F170C945D320C94000081E00895089585
:100BB0000C94AF070C94D5050C94D7050E94272EF2
:100BC000811105C010920203109201030DC081E251
:100BD00090E00090030302C0880F991F0A94E2F787
:100BE000909302038093010382E08093000380913D
:100BF0006F00826080936F00089590916F0081E094
:100C0000911101C080E008950E94272E23E030E07A
:100C1000281B3109220F209304030895282F2F98B1
:100C200080918000211108C0877F809380001092FE
:100C30008D0010928C001BC0886080938000233050
:100C400019F48FEF9FEF0FC083E090E0821B9109B2
:100C5000880F991F2FEF3FEFA90102C056954795C6
:100C60008A95E2F7CA0190938D0080938C000C94D2
:100C70000406CF93C82F0E94FD05409103038823EB
:100C800029F090916F009D7F90936F00C0930303B4
:100C90008823D1F0209101033091020302C03695E0
:100CA00027954A95E2F72F733327C90102C0880FB1
:100CB000991FCA95E2F790930203809301038091F4
:100CC0006F00826080936F00CF9108950E940406A8
:100CD00084E080930303109200030895279A2F98CD
:100CE0008FEF9FEF90938700809386008AE0809338
:100CF000800089E1809381000E94902D0C9466060B
:100D00000E946E066E9A769A0C9497071F920F9225
:100D10000FB60F9211242F933F938F939F93EF93CE
:100D2000FF93E0910103F0910203CF0101969093AC
:100D30000203809301030090030302C0F695E79538
:100D40000A94E2F7EF7380910003823019F4E032E5
:100D500051F404C0813039F4EF3329F480916F00ED
:100D60008D7F80936F00F0E0E855FE4FE49121E025
:100D700031E0E29FC001E39F900D11240090040335
:100D800002C0969587950A94E2F790938D00809320
:100D90008C00FF91EF919F918F913F912F910F9038
:100DA0000FBE0F901F901895CF93DF93EC010E9418
:100DB0002E29BE0180E090E0DF91CF910C94232595
:100DC0000F931F93462F50E04E30510508F0AAC0F4
:100DD000DC01FA01EA5AFF4F0C94213212968C91F1
:100DE000882309F49FC000E010E0980140E064E02F
:100DF00070E080ED91E00E94591381E090E011C015
:100E000012968C91882309F48DC000E010E09801BF
:100E100040E066E070E080E691E00E94591382E0D5
:100E200090E00E94D4067EC012968C91882309F42B
:100E300079C000E010E0980140E068E070E080E9EF
:100E400091E00E94591384E090E0EBCF12968C91D0
:100E5000882311F083E007C083E013C012968C91C1
:100E6000882371F084E00E94A02582E00E94390668
:100E70000E94DE0540E164E083E00E94BE0D52C0A6
:100E800084E00E94C125F6CF12968C91882331F020
:100E900085EE0E94B81D0E94E72D44C085EE0E9499
:100EA000801E40C012968C918823E1F10E940E0FA3
:100EB00000E010E0980140E066E070E080E391E03F
:100EC0000E94591384E00E94C12583E00E94C1253D
:100ED00080E10E94C12585E00E94A0250E941B2977
:100EE000811102C00E94F7280E94332990E090935C
:100EF0005D0480935C04806880935C040E943729C1
:100F000011C012968C91882369F000E010E09801DE
:100F100040E066E070E080E091E00E94591385E0D7
:100F20000E94C12580E090E01F910F9108950F93DA
:100F30001F932FEF89EF90E0215080409040E1F720
:100F400000C0000000E010E0980140E065E070E0C3
:100F500080EF91E00E9459131F910F9108958091A5
:100F60001003882309F45AC080910E0390910F0357
:100F70000E946B288D3291400CF450C010921003E7
:100F80000E9414088091080390910903099781F445
:100F900080910A0390910B03892B51F480910C03EB
:100FA00090910D03892B21F48AE592E00E941508A7
:100FB0008091080390910903049791F480910A03AA
:100FC00090910B03469761F480910C0390910D036F
:100FD000892B31F48BE00E94B81D8BE00E94801EAB
:100FE00080910803909109030497C1F480910A034A
:100FF00090910B03469791F480910C0390910D030F
:10100000079761F483EE0E94B81D86E10E94B81D27
:1010100086E10E94801E83EE0C94801E089581E07C
:1010200008950C940F08089508950F931F93CF937C
:101030008C01F80124912223F9F030E0F901E85BFA
:10104000F74FC491F901E853F74F2491222359F047
:1010500081EE0E94B81D8C2F0E94B81D8C2F0E941B
:10106000801E81EE04C08C2F0E94B81D8C2F0E9420
:10107000801E0F5F1F4FDDCFCF911F910F910895FD
:101080000C94800680915503882309F448C0809110
:10109000110390911203009779F40E945F289093B6
:1010A0001203809311038091130390E0009771F471
:1010B0008091140390E00AC00E946B2820911802CE
:1010C000309119022817390740F329C00197880F7A
:1010D000991F880F991FFC01EB5EFC4F60817181A5
:1010E000828193810E94410FE091130384E0E89F85
:1010F000F0011124EB5EFC4F60817181828193814C
:101100004FE050E00E94F9128091130390E00196A5
:101110006091140370E00E940D32809313030C94CD
:10112000D805109257030C940E0F0895089581E08E
:10113000809357030C949608089508958F929F9278
:10114000AF92BF92EF92FF920F931F93CF93DF93D3
:10115000CDB7DEB7A3970FB6F894DEBF0FBECDBFF5
:101160007C01FC0100811181C8010E945C26B8014C
:101170000E94A00A8C01B7010E941108882309F47B
:10118000CCC10032F0E51F0741F4F70182818823CA
:1011900009F458C00E94F013C0C10132F0E51F07E6
:1011A00041F4F7018281882309F44CC00E94F913AD
:1011B000B4C10232F0E51F0751F4F70182818823A0
:1011C00009F440C00E94EC138111F0CFE3CF033249
:1011D000F0E51F0739F4F7018281882399F10E9415
:1011E00097089BC10432F0E51F0739F4F7018281AB
:1011F000882341F10E94910890C10532F0E51F0754
:1012000049F4F70182818823E9F080915703811125
:10121000F1CFE5CF0632F0E51F0739F4F7018281FF
:10122000882381F00E9400140AC00732F0E51F07EE
:1012300049F4F7018281882329F00E940B140E944F
:101240009D086BC180915703811105C0F701828110
:101250008111CFC018C1003E110579F4F7018281D8
:10126000882309F44DC00E940E0F81E0809356033D
:10127000109255031092140350C1023E110559F407
:10128000F70182818823E1F10E940E0F109256032C
:101290001092550342C1033E110591F4F70182817A
:1012A000882371F10E940E0F1092560381E0809303
:1012B00055031092130310921203109211032DC1C3
:1012C0000235110559F4F7018281882309F425C1FB
:1012D00080911802909119020A970DC001351105ED
:1012E00079F4F7018281882309F417C180911802EB
:1012F000909119020A9690931902809318020DC1D9
:1013000040911C0283E2E7E3F2E0DE0111960190D6
:101310000D928A95E1F7F701808121E030E02C0FF2
:101320003D1F280F311DC90120911A0230911B0267
:10133000FC01E20FF31F6081772767FD7095640F52
:10134000711D882777FD8095982F0E942F2F20E010
:1013500030E040E451E40E94942E4B015C01F7011F
:10136000218184E090E0821B9109BC01882777FDF0
:101370008095982F0E942F2F9B01AC01C501B401CD
:101380000E942C2E9B01AC0160E070E080E090E4B4
:101390000E94A23020E030E04CED50E40E943F304B
:1013A0004B015C01F70182818823D1F04FE050E0CE
:1013B000C501B4010E94F912809156038823A1F05F
:1013C0008091140324E0829FF0011124EB5EFC4F16
:1013D00080829182A282B3828F5F8093140304C0C3
:1013E000C501B4010E94410F0F3F110508F02ECF37
:1013F00094C08091100381111FC0043130E51307A0
:1014000009F051C00E94130881E0809310030E94EC
:101410005F2890930F0380930E031092070310929E
:1014200009031092080310920B0310920A03109202
:101430000D0310920C0371C080910E0390910F0365
:101440000E946B28883C910570F480910703E82F77
:10145000F0E0EE0FFF1FE85FFC4F118300838F5F0A
:10146000809307035AC0043880E5180721F0053837
:10147000104501F13AC0F7018281882341F01092B2
:10148000050382E01EC0043830E5130759F580914A
:101490000503811106C086E20E94B81D86E20E9403
:1014A000801E82E01CC00438F0E51F0741F30538B8
:1014B0001045D9F4F7018281882331F01092060398
:1014C00080E20E94CF1E29C080910603811106C0D0
:1014D00087E20E94B81D87E20E94801E80E20E947F
:1014E000D61E1BC00538104529F381E08093050303
:1014F00080930603C701A3960FB6F894DEBF0FBE14
:10150000CDBFDF91CF911F910F91FF90EF90BF90D2
:10151000AF909F908F900C94DA0580E0A3960FB661
:10152000F894DEBF0FBECDBFDF91CF911F910F9119
:10153000FF90EF90BF90AF909F908F900895089587
:101540009CE0799FF001112490E3899FE00DF11D4B
:101550001124E60FF11DEE0FFF1FE851FE4F85919C
:1015600094910895880F991FFC01E859FF4F8591C8
:1015700094910895880F991FFC01E851FE4F8591C1
:10158000949108950F931F93CF93DF93EC018115EE
:1015900021E39207A0F5C11580E3D80708F0D7C072
:1015A000C83ED105D8F4C03ED10508F007C2C83AFC
:1015B000D10578F4C53AD10508F06AC0C130D1052B
:1015C00009F463C008F4F7C1C430D10508F0F6C1CE
:1015D000F2C1CB3BD10508F466C0EDC1C11590E264
:1015E000D90708F0AFC0C11521E0D20708F0E6C165
:1015F000C03FD10508F4DFC18E0110651FC2C0389D
:1016000080E5D80700F5C03790E5D90708F0A3C0FA
:10161000C11520E5D20709F4ACC050F4CE019054B6
:1016200080319F4008F0C7C1DF708E01106A06C28A
:10163000C13080E5D80709F4AEC0C43190E5D907C0
:1016400008F4AFC0B8C1C33820E5D20709F48EC092
:1016500050F4C13890E5D90709F482C008F083C07E
:1016600000E011EDEBC1C03181E5D80708F4A3C15A
:10167000C11597E5D90708F436C1CE0190578115F9
:10168000904108F098C1DF7093C101E010E0D6C12D
:10169000C53AD10509F494C1C63AD10509F093C100
:1016A00002E810E4CBC1C83AD10509F48FC1C93AA8
:1016B000D10509F48EC1CA3AD10509F48DC1CB3ADE
:1016C000D10509F48CC1CC3AD10509F48BC1CD3ACE
:1016D000D10509F48AC1C03BD10509F489C1CE3ACC
:1016E000D10509F488C1CF3AD10509F487C1C13BBE
:1016F000D10509F486C1C23BD10509F485C1C33BBC
:10170000D10509F484C1C43BD10509F483C1C53BAB
:10171000D10509F482C1C63BD10509F481C1C73B9B
:10172000D10509F480C1C83BD10509F47FC1C93B8B
:10173000D10509F47EC1CA3BD10509F47DC100E0A1
:1017400014E47CC1CE019F700E94BA0A78C1DD27E3
:101750008E01106C73C1CF70DD278E01146D6EC1C8
:1017600000E010ED6BC100E012ED68C100E013ED88
:1017700065C10E9463210E940E0F0E9495088FEFA1
:1017800094E32CE0815090402040E1F700C000003D
:101790000E94BA2853C18091320481608093320440
:1017A0004DC10E941B29811102C00E94F7280E948E
:1017B000332990E090935D0480935C04C23080E50F
:1017C000D80721F480915C04816086C0C43090E524
:1017D000D90721F480915C0482607EC0C63020E588
:1017E000D20721F480915C04846076C0C83080E523
:1017F000D80719F480915C0427C0CA3090E5D90756
:1018000021F480915C04806167C0CC3020E5D20770
:1018100021F480915C0480625FC0CE3080E5D807FF
:1018200021F480915C04806457C0C03190E5D907F1
:1018300021F480915C0480684FC0C23120E5D2075A
:1018400029F480915C048460886046C0C33080E5E0
:10185000D80721F480915C048E7F3EC0C53090E5AE
:10186000D90721F480915C048D7F36C0C73020E514
:10187000D20721F480915C048B7F2EC0C93080E5B3
:10188000D80719F480915C0426C0CB3090E5D907C5
:1018900021F480915C048F7E1FC0CD3020E5D207FB
:1018A00021F480915C048F7D17C0CF3080E5D8078C
:1018B00021F480915C048F7B0FC0C13190E5D90782
:1018C00021F480915C048F7707C0C331D04531F497
:1018D00080915C048B7F877F80935C0480915C04A3
:1018E0000E943729ABC08D2F99278F70992781309F
:1018F0009105D9F49E012370332702C0880F991FE8
:101900002A95E2F79C688E0144E0000F111F4A956A
:10191000E1F700271370802B912B53E0CC0FDD1FD4
:101920005A95E1F7C076DD272FC08230910531F45A
:10193000DC2FCC278E01016F106A80C083309105A7
:1019400069F4CE018370992701E010E002C0000F16
:10195000111F8A95E2F7C8019C680FC08430910579
:10196000B9F4CE018370992701E010E002C0000FA6
:10197000111F8A95E2F7C8019A6823E0CC0FDD1F9A
:101980002A95E1F7C07ED7708C010C2B1D2B56C019
:101990008530910531F4DC2FCC278E01046F106A5D
:1019A0004DC0069709F04AC0CF71DD27DC2FCC2748
:1019B0008E01106243C000E010E040C08E013EC0C6
:1019C00001E810E43BC003E810E438C002EE14E480
:1019D00035C009EE14E432C00AEE14E42FC005EB62
:1019E00014E42CC006EB14E429C007EB14E426C071
:1019F0000CEC14E423C00DEC14E420C003E815E45F
:101A00001DC00AE815E41AC002E915E417C004E98C
:101A100015E414C001E216E411C003E216E40EC09E
:101A200004E216E40BC005E216E408C006E216E480
:101A300005C007E216E402C00AE216E4C801DF911D
:101A4000CF911F910F9108959CE0799FF00111248F
:101A500090E3899FE00DF11D1124E60FF11DEE0FBB
:101A6000FF1FE851FE4F85919491803E9105E0F46F
:101A7000803C910558F58133910509F46FC048F415
:101A80008932910509F463C08A32910509F46DC069
:101A900072C089339105E9F082389105D1F0853320
:101AA000910509F44DC067C0833E910581F138F47A
:101AB000803E9105B9F0823E9105D9F05CC0863E2A
:101AC000910561F1873E9105A1F155C00E94B20ACE
:101AD000089520915C0420FD02C021FF4CC080EEDF
:101AE00090E049C080915C0480FFF9CF89E390E0E9
:101AF00042C080915C0482FF0EC080915C0484FF30
:101B000003C080E090E037C083EE90E034C0809165
:101B10005C0482FFF2CF82EE90E02DC080915C04E5
:101B200083FF0BC080915C0484FDEBCF87EE90E0D7
:101B300022C080915C0483FFF5CF86EE90E01BC04D
:101B400080915C0485FF07C089E290E014C0809119
:101B50005C0485FFF9CF85E390E00DC080915C04C3
:101B600086FF07C08AE290E006C080915C0486FF91
:101B7000F9CF81E390E00E94C20A0895CF92DF92EC
:101B8000EF92FF920F931F9301E010E020E030E00E
:101B90006801790104C0CC0CDD1CEE1CFF1C8A9589
:101BA000D2F704C0000F111F221F331F6A95D2F70E
:101BB0000C291D292E293F29C0901504D090160408
:101BC000E0901704F0901804C022D122E222F32200
:101BD000842FC016D106E206F30641F41F910F913F
:101BE000FF90EF90DF90CF900C94A0251F910F9164
:101BF000FF90EF90DF90CF900C94C1250C94DC0502
:101C0000E82FF0E0E257FD4F8081E82FEF70F0E021
:101C100082958F7021E030E0A90102C0440F551F6A
:101C20008A95E2F740A308950F931F93CF93DF9314
:101C300085B7806885BF85B7806885BFC3E0D0E081
:101C400001E010E0FE01E257FD4F8081E82FEF70C8
:101C5000F0E021A182958F70A80102C0440F551FAA
:101C60008A95E2F7CA01822B81A38C2F0E94000E75
:101C7000219740F78BE090E061E070E0FC01EE57C7
:101C8000FD4F2081E22FEF70F0E042A122952F70EE
:101C9000DB0102C0AA0FBB1F2A95E2F79D01242B8E
:101CA00022A3019758F7DF91CF911F910F910C94C8
:101CB0004008EF92FF920F931F93CF93DF9300E6BC
:101CC00013E0C3E0EE24E394F12CD5E08C2F0E94C6
:101CD000000E8BE090E040E050E0FC01EE57FD4F3D
:101CE0006081E62FEF70F0E020A130E062956F7028
:101CF00002C0359527956A95E2F720FD09C0970146
:101D0000082E02C0220F331F0A94E2F7422B532BF6
:101D1000019718F7F801929182918F018417950726
:101D200021F051834083D0931D028C2F0E94000E1E
:101D3000C15060F680911D0287FD2CC081508093B8
:101D40001D028F3F39F08FE99FE00197F1F700C046
:101D5000000020C080915E0390915F039093670321
:101D60008093660380915C0390915D03909365037B
:101D70008093640380915A0390915B039093630373
:101D8000809362038091580390915903909361036B
:101D9000809360030E94420881E0DF91CF911F9100
:101DA0000F91FF90EF900895E82FF0E0EE0FFF1FE6
:101DB000E05AFC4F80819181089508950F931F93FD
:101DC000CF9308E613E0C0E0F801929182918F0171
:101DD0000E94D727C80FF3E000361F07A9F78C2F02
:101DE000CF911F910F9108950E941B29811102C06C
:101DF0000E94F7280E944529809347043E9A8091CB
:101E000071008D7F8093710082E0809390008AE161
:101E10008093910081E080936A03089580916A0322
:101E2000811102C00E94F40E1092BA031092B903FD
:101E3000809171008D7F80937100809190008F73ED
:101E40008093900010927C0310927B031092B30356
:101E50001092B4031092B5031092B6031092B2031D
:101E60001092B103E1E9F3E0A1E8B3E0119211921D
:101E7000119211921D921D9283E0E13BF807B1F798
:101E80000895CF92DF92EF92FF920F931F93CF931B
:101E9000DF9320917B03222309F484C06B017C0132
:101EA00080916A03811102C00E94F40E01EB13E0DD
:101EB000C7E0D0E0A7019601F8019291829172915A
:101EC00062918F010E94902E811131C0FE01EE0FB0
:101ED000FF1FEE0FFF1FEF56FC4F10821182128280
:101EE0001382DE01AA0FBB1FAF57BC4F11961C9285
:101EF0001E92C730D105E9F0219644815581668153
:101F000077814083518362837383148215821682A2
:101F1000178212968D919C91139711969C938E9394
:101F200013961C921E92129734961296E2CF219726
:101F300008F68091B9039091BA03019797FD05C007
:101F40009093BA038093B90304C01092BA0310921D
:101F5000B9038091B9039091BA032091B7033091EE
:101F6000B8032817390724F01092B8031092B7036A
:101F7000892BC1F4809171008D7F809371008091D5
:101F800090008F73809390001092B3031092B4036B
:101F90001092B5031092B6031092B2031092B103DF
:101FA00010927B03DF91CF911F910F91FF90EF90E3
:101FB000DF90CF9008951F920F920FB60F921124C9
:101FC0004F925F926F927F928F929F92AF92BF9249
:101FD000CF92DF92EF92FF922F933F934F935F93B5
:101FE0006F937F938F939F93AF93BF93CF93DF9321
:101FF000EF93FF9380917B03882309F49BC1C091E9
:10200000B903D091BA031C161D060CF093C1409081
:102010006B0350906C0360906D0370906E0320E032
:1020200030E0A901C301B2010E943B3018160CF048
:1020300065C0C130D10509F452C08091B7039091B9
:10204000B803BE010E940D327C019093B8038093C7
:10205000B70380907D0390907E03A0907F03B090A3
:10206000800320E030E040E85FE3C501B4010E9456
:102070002C2E60937D0370937E0380937F03909357
:102080008003F701EE0FFF1FEE0FFF1FEF56FC4F0F
:10209000A301920160817181828193810E94942EBB
:1020A00020E030E040E05EE30E943F309B01AC0165
:1020B000C501B4010E943B3018168CF4C70101968B
:1020C000BE010E940D329093B8038093B703109223
:1020D0007D0310927E0310927F0310928003E091A3
:1020E000B703F091B803EE0FFF1FEE0FFF1FEF567F
:1020F000FC4F6081718182819381D0C0C090B30315
:10210000D090B403E090B503F090B60320E030E047
:10211000A901C701B6010E94902E2197882309F4D6
:10212000A2C0FE01EE0FFF1FEE0FFF1FEF56FC4F88
:1021300080809180A280B380A5019401C701B6017F
:102140000E94902E87FF31C0A501940160E070E0ED
:102150008CED93EC0E94942E20E030E040E451E4BA
:102160000E94942E20E030E040E05FE30E943F3088
:102170009B01AC0160E070E080E090E40E94A2303E
:102180009B01AC01C501B4010E943F309B01AC0131
:10219000C701B6010E94902E87FF07C0A7019601D4
:1021A00060E070E08CED93E439C0A5019401C701B3
:1021B000B6010E943B3018160CF055C0A5019401E1
:1021C00060E070E08CED93E40E94942E20E030E01B
:1021D00040E451E40E94942E20E030E040E05FE3D0
:1021E0000E943F309B01AC0160E070E080E090E431
:1021F0000E94A2309B01AC01C501B4010E943F3096
:102200009B01AC01C701B6010E943B3018165CF57A
:10221000A701960160E070E08CED93EC0E94942E93
:1022200020E030E040E451E40E94942E20E030E0D1
:1022300040E05FE30E943F309B01AC0160E070E052
:1022400080E090E40E94A2309B01AC01C701B6017E
:102250000E943F306093B3037093B4038093B5033F
:102260009093B60313C0FE01EE0FFF1FEE0FFF1F8A
:10227000EF56FC4F80819181A281B3818093B3039B
:102280009093B403A093B503B093B6036091B303E6
:102290007091B4038091B5039091B60320916803C7
:1022A000309169032F3F4FEF340731F02F5F3F4FDD
:1022B00030936903209368030E9416146B017C011C
:1022C00020E034E244EF51E40E94902E87FF08C0E2
:1022D00086EFC82E88E2D82E84EFE82E81E4F82E0F
:1022E00020E030E040E051E4C701B6010E943F30F9
:1022F0009B01AC0160E074E284E79BE40E94942EB1
:102300006B017C010E94012F7093970060939600EF
:1023100020911E0230911F02409120025091210213
:10232000C701B6010E943F300E94012F70939900AF
:102330006093980080917C03882309F433C1C09096
:102340007703D0907803E0907903F0907A0320E04F
:1023500030E0A901C701B6010E943B301816D4F540
:1023600080916803909169038F3F2FEF920729F0C6
:1023700001969093690380936803C701B6010E9498
:10238000161420E030E040E051E40E943F309B0111
:10239000AC0160E074E284E79BE40E94942E6B0140
:1023A0007C010E94012F709397006093960020910A
:1023B0001E0230911F024091200250912102C7015C
:1023C000B6010E943F300E94012F709399006093E4
:1023D000980008C0109297001092960010929900F1
:1023E0001092980060917103709172036F5F7F4F3C
:1023F000709372036093710320919600309197005F
:1024000080E090E0232BF1F0C0919600D0919700EE
:102410000E942D2F6B017C01BE0180E090E00E94A4
:102420002D2F9B01AC016091730370917403809117
:102430007503909176030E94942E20E03FEF4FE7C2
:1024400057E410C00E942D2F6B017C0120E030EE7C
:102450004FEF54E46091730370917403809175039E
:10246000909176030E943F309B01AC01C701B601F9
:102470000E943B3087FD96C080916F038F5F8093F1
:102480006F0390E020914304309144048217930736
:10249000A0F080914E04882319F010926F030DC0B4
:1024A000809171008D7F80937100809190008F7377
:1024B0008093900010927C037DC080917003C09146
:1024C0006F03811128C0C0904804D0904904E09067
:1024D0004A04F0904B0420E030E0A901C701B601A6
:1024E0000E943B301816BCF481E080937003109278
:1024F0007703109278031092790310927A03C092B6
:102500007303D0927403E0927503F0927603C15086
:10251000C0936F0343C0109270031092690310922E
:102520006803E0914504F091460448E0C49FE00D43
:10253000F11D112480819181A281B3818093770361
:1025400090937803A0937903B0937A0320E030E06E
:1025500040E85EE364817581868197810E943F3007
:102560006B017C0180912202682F70E080E090E096
:102570000E942D2F20E030E048EC52E40E94942E7F
:102580009B01AC01C701B6010E943F306093730309
:102590007093740380937503909376031092720383
:1025A000109271038091470480FD04C010927C0357
:1025B00010927B03FF91EF91DF91CF91BF91AF918B
:1025C0009F918F917F916F915F914F913F912F914B
:1025D000FF90EF90DF90CF90BF90AF909F908F9043
:1025E0007F906F905F904F900F900FBE0F901F9055
:1025F0001895CF92DF92EF92FF92CF93DF936B010A
:102600007C01EA0180916A03811102C00E94F40EEC
:102610008091470480FF46C08091B9039091BA032E
:1026200008970CF03FC0809171008D7F80937100FE
:1026300080917C0381110E940E0F81E080937B03C7
:10264000109269031092680320E030E0A901C701ED
:10265000B6010E943B301816DCF48091B9039091CA
:10266000BA03FC01EE0FFF1FEE0FFF1FEF56FC4FEA
:10267000C082D182E282F382FC01EE0FFF1FEF578E
:10268000FC4FD183C08301969093BA038093B90322
:1026900080917100826080937100809190008068C9
:1026A00080939000DF91CF91FF90EF90DF90CF90DB
:1026B00008958F929F92AF92BF92CF92DF92EF9246
:1026C000FF920F931F93CF93DF93EC017B01D42EE6
:1026D0004801590180916A03811102C00E94F40EE1
:1026E0008091470480FF6BC0809171008D7F809343
:1026F000710080917B0381110E940E0F81E0809315
:102700007C03D0934604C0934504F0924404E092C5
:102710004304D0924E048092480490924904A092BF
:102720004A04B0924B0410927D0310927E031092E3
:102730007F031092800310926F0388819981AA8190
:10274000BB818093770390937803A0937903B09330
:102750007A0320E030E040E85EE36C817D818E8189
:102760009F810E943F306B017C0180912202682F83
:1027700070E080E090E00E942D2F20E030E048ECF7
:1027800052E40E94942E9B01AC01C701B6010E9445
:102790003F30609373037093740380937503909339
:1027A000760310927203109271038091710082601F
:1027B0008093710080919000806880939000DF91F9
:1027C000CF911F910F91FF90EF90DF90CF90BF902E
:1027D000AF909F908F9008958091470481700895E5
:1027E000809147048160809347040E9449290C949A
:1027F0009C08809147048E7F809347040C9449295C
:102800008091BB0390E0019666E070E00E940D327B
:102810008093BB0308958091BB0390E0019766E02D
:1028200070E00E940D328093BB0308958F929F92B7
:10283000AF92BF92CF92DF92EF92FF920F931F93CE
:10284000CF93DF936B017C01C0916803D091690342
:10285000BE0180E090E00E942D2F4B015C01A7019A
:10286000960160E070E08CE594E40E94942E9B0158
:10287000AC01C501B4010E943F300E94012F20919C
:10288000BB03233009F473C028F4222351F0213014
:10289000E9F02CC1243009F4A0C0253009F4E0C0CF
:1028A00025C180E090E0A0E0BFE380931E029093FA
:1028B0001F02A0932002B093210210926B0310928A
:1028C0006C0310926D0310926E0310C110926B0393
:1028D00010926C0310926D0310926E0364317105B7
:1028E00040F46A30710560F520E030E040E85EE3D6
:1028F0002BC0693C710508F0AAC080E090E00E94FE
:102900002D2F20E030E040EA51E40E942B2E20E001
:1029100030E044E353E40E94942E9B01AC010E94FA
:102920003F3020E030E040E05EE30E943F309B011A
:10293000AC0160E070E080E09EE30E942B2E44C07A
:1029400020E030E040E05FE3C701B6010E943F3085
:102950006B017C0180E090E0A0E0BEE380931E026A
:1029600090931F02A0932002B0932102BFC0109247
:102970006B0310926C0310926D0310926E034AE089
:10298000469F9001479F300D1124C90168EB7BE001
:102990000E94F931BC016C5D754077FF03C07195F1
:1029A00061957109882777FD8095982F0E942F2FB8
:1029B0002EE333EC4EE259E30E943F3020E030E05A
:1029C00040EC5EE30E942C2E60931E0270931F0267
:1029D000809320029093210289C010926B03109281
:1029E0006C0310926D0310926E03CE0183709927D1
:1029F000892BE1F0BE016170772780E090E00E94B2
:102A00002D2F20E030E040E05EE30E943F3020E0E8
:102A100030E040E45FE30E942C2E60931E0270932E
:102A20001F0280932002909321020CC080E090E06E
:102A3000A0E0BFE380931E0290931F02A0932002A8
:102A4000B0932102C770DD27CD2B09F04FC0109243
:102A50001E0210921F02109220021092210246C004
:102A600010926B0310926C0310926D0310926E0320
:102A700000E010E020E03FE300931E0210931F02ED
:102A800020932002309321026739710578F180E0AC
:102A900090E00E942D2F20E030E047E153E40E94B7
:102AA0002B2E20E030E04AE754E40E94942E20E0F0
:102AB00030E048E452E40E943F3020E030E040EA59
:102AC00051E40E94712F0E94FC2E660F771F660F43
:102AD000771FFB01EE56FD4F2081318142815381EA
:102AE000C701B6010E943F306B017C01C701B601EE
:102AF000DF91CF911F910F91FF90EF90DF90CF90DA
:102B0000BF90AF909F908F9008958091CC030895CF
:102B1000CF93DF9300D01F92CDB7DEB79C01809199
:102B20005304843019F593E099833B832A8390936F
:102B3000E9008FEF9091E800815095FD06C095ED7A
:102B40009A95F1F700008111F5CF8091E80085FF9B
:102B50000DC040E050E063E070E0CE0101960E94BD
:102B6000E9178091E8008E778093E8000F900F902E
:102B70000F90DF91CF910895CF93DF9300D01F92F4
:102B8000CDB7DEB720915304243021F522E029830C
:102B90009B838A8383E08093E9008FEF9091E80024
:102BA000815095FD06C095ED9A95F1F700008111D1
:102BB000F5CF8091E80085FF0DC040E050E063E074
:102BC00070E0CE0101960E94E9178091E8008E77AF
:102BD0008093E8000F900F900F90DF91CF910895B0
:102BE000209153042430F1F422E02093E9002FEFE8
:102BF0003091E800215035FD06C035ED3A95F1F7EA
:102C000000002111F5CF2091E80025FF0BC040E026
:102C100050E065E070E00E94E9178091E8008E774F
:102C20008093E8000895CF93DF93EC0190915304D3
:102C3000943009F046C080912D028823D9F080910C
:102C40002E028823B9F09093E9008FEF9091E8006D
:102C5000815095FD06C095E19A95F1F7000081112C
:102C6000F5CF8091E80085FF2CC040E050E060E1A6
:102C700070E017C081E08093E9008FEF9091E80049
:102C8000815095FD06C095ED9A95F1F700008111F0
:102C9000F5CF8091E80085FF14C040E050E068E087
:102CA00070E0CE010E94E9178091E8008E77809352
:102CB000E80080E1FE01ACEBB3E001900D928A9553
:102CC000E1F7DF91CF91089580915204811109C0FD
:102CD0000E947E190E94DB198091E200846080933B
:102CE000E2000895109252040895089508950C94F6
:102CF000222842E061EC81E00E94F81842E061EC99
:102D000082E00E94F81842E061EC83E00E94F8182B
:102D100042E161EC84E00C94F81880915504833012
:102D200009F455C030F4813071F0823009F48EC05E
:102D300008958A3009F47AC08B3009F460C0893074
:102D400009F09CC020C080915404813A09F096C0DB
:102D50008091E800877F8093E800809158049091EB
:102D60005904892B21F460E18CEB93E003C060E00F
:102D700080E090E070E00E9434188091E8008B774A
:102D80008093E800089580915404813209F076C060
:102D90008091580490915904009719F0039709F015
:102DA0006DC08091E800877F8093E8008091E80003
:102DB00082FD05C0809153048111F8CF5FC08091DE
:102DC000F1008093CC038091E8008B7753C0809111
:102DD0005404813A09F052C08091580490915904EA
:102DE000892B09F04BC08091E800877F8093E80031
:102DF0008091E80080FFFCCF80912D0236C0809149
:102E000054048132D9F58091580490915904892B4A
:102E1000A9F58091E800877F8093E8000E942D1932
:102E20008091560480932D020C9463218091540468
:102E3000813221F58091E800877F8093E8000E942D
:102E40002D19809157048093CD03089580915404E7
:102E5000813AA1F48091E800877F8093E800809117
:102E6000E80080FFFCCF8091CD038093F10080913A
:102E7000E8008E778093E8000C942D19089584B7AC
:102E8000877F84BF88E10FB6F8948093600010922A
:102E900060000FBE90E080E80FB6F8948093610068
:102EA000909361000FBE0E94D01C0E947E190E9468
:102EB000DB198091E20084608093E20078940E94A4
:102EC000611C0E94D21C83E292E00E947C1C8091D3
:102ED0005304853069F40E94E327809151048823CC
:102EE000B1F30E941128882391F30E94D317EFCFEA
:102EF0000E94DA1CECCF292F332723303105C9F08B
:102F000064F42130310581F02230310509F043C0ED
:102F10008DE690E024EA39E042C021323105F1F03B
:102F20002232310541F137C082E190E021E13AE0FF
:102F300036C099278130910541F08230910541F0EA
:102F4000892B49F5E0EAF9E005C0E2E7F9E002C0C3
:102F5000E8E4F9E0849190E09F0121C06430D8F466
:102F6000E62FF0E0EE0FFF1FE251FD4F208131818F
:102F700089E090E014C0643070F470E0FB01EE0F63
:102F8000FF1FEA51FD4F20813181FB01EE51FD4FC2
:102F9000808190E004C080E090E020E030E0FA0121
:102FA00031832083089580E189BD82E189BD09B420
:102FB00000FEFDCF8091D8008F7D8093D800809156
:102FC000E00082608093E0008091E00081FDFCCF12
:102FD0000895CF92DF92EF92FF920F931F93CF93BA
:102FE000DF93EC018B016A010E944C19811133C0FF
:102FF000C114D10439F0F60180819181081B190BAD
:10300000C80FD91FE12CF12C0115110519F1809180
:10301000E80085FD16C08091E8008E778093E80077
:10302000C114D10449F0F60180819181E80EF91EA6
:10303000F182E08285E00FC00E944C19882321F3C1
:103040000AC089918093F10001501109FFEFEF1A36
:10305000FF0ADACF80E0DF91CF911F910F91FF90AF
:10306000EF90DF90CF90089520915A0430915B0447
:103070002617370748F06115710539F42091E800EB
:103080002E772093E80001C0B90140E06115710579
:10309000A9F120915304222309F443C0253009F4F7
:1030A00042C02091E80023FD40C02091E80022FDAD
:1030B00032C02091E80020FFE9CF4091F300209139
:1030C000F20030E0342BFC01CF016115710559F09D
:1030D0002830310540F481918093F10061507109ED
:1030E0002F5F3F4FF1CF41E02830310509F040E03C
:1030F0002091E8002E772093E800C8CF4111C9CF76
:103100000AC080915304882361F0853061F080917A
:10311000E80083FD0AC08091E80082FFF2CF80E0E2
:10312000089582E0089583E0089581E00895209154
:103130005A0430915B042617370748F06115710572
:1031400039F42091E8002E772093E80001C0B901FE
:10315000FC0120E06115710591F1809153048823F1
:1031600009F440C0853009F43FC08091E80083FD38
:103170003DC08091E80082FD2FC08091E80080FF73
:10318000E9CF2091F3008091F20090E0922B61153D
:10319000710559F08830910540F424912093F10095
:1031A0003196615071090196F2CF21E0089709F03C
:1031B00020E08091E8008E778093E800CBCF21114A
:1031C000CCCF0AC080915304882361F0853061F030
:1031D0008091E80083FD0AC08091E80082FFF2CF71
:1031E00080E0089582E0089583E0089581E00895E5
:1031F000982F973058F59093E900981739F070910F
:10320000EC002091ED005091F00003C0242F762FA8
:1032100050E021FF19C03091EB003E7F3093EB006E
:103220003091ED003D7F3093ED003091EB00316047
:103230003093EB007093EC002093ED005093F0007E
:103240002091EE0027FF07C09F5FD3CF8F70809340
:10325000E90081E0089580E008958091540487FF9B
:1032600011C08091E80082FD05C080915304811156
:10327000F8CF11C08091E8008B770BC08091530488
:10328000882349F08091E80080FFF8CF8091E80022
:103290008E778093E80008952091E4003091E50056
:1032A00095E64091EC00842F817040FF22C0809110
:1032B000E80080FD1CC080915304882391F0853084
:1032C00091F08091EB0085FD10C04091E400509199
:1032D000E5004217530729F39A01915011F784E052
:1032E000089582E0089583E0089581E0089580E0E4
:1032F00008954091E80042FFDECF08950E94EC1946
:103300000E94F419E0EEF0E0808181608083E8EDB6
:10331000F0E080818F77808319BCA7EDB0E08C91BD
:103320008E7F8C9380818F7E8083109252040895CB
:103330000F931F93CF93DF930E94EC190E94F4190F
:10334000C8EDD0E088818F77888388818068888302
:1033500088818F7D888319BC1092530410924F048A
:10336000109251041092500400EE10E0F801808198
:103370008B7F808388818160888342E060E080E089
:103380000E94F818E1EEF0E080818E7F8083E2EE0B
:10339000F0E0808181608083808188608083F80193
:1033A00080818E7F8083888180618883DF91CF9147
:1033B0001F910F910895E8EDF0E080818F7E80836A
:1033C000E7EDF0E080818160808384E082BF81E06E
:1033D000809352040C949819E8EDF0E080818E7F80
:1033E00080831092E20008951092DA001092E100BA
:1033F00008951F920F920FB60F9211242F933F93AF
:103400004F935F936F937F938F939F93AF93BF93EC
:10341000EF93FF938091E10082FF0BC08091E20067
:1034200082FF07C08091E1008B7F8093E1000E94C2
:10343000601C8091DA0080FF1FC08091D80080FF5F
:103440001BC08091DA008E7F8093DA008091D900D2
:1034500080FF0DC080E189BD82E189BD09B400FE15
:10346000FDCF81E0809353040E94641605C019BC0F
:10347000109253040E9472168091E10080FF19C0DF
:103480008091E20080FF15C08091E2008E7F8093E2
:10349000E2008091E20080618093E2008091D80098
:1034A00080628093D80019BC85E0809353040E9409
:1034B00076168091E10084FF30C08091E20084FFA5
:1034C0002CC080E189BD82E189BD09B400FEFDCF39
:1034D0008091D8008F7D8093D8008091E1008F7E0D
:1034E0008093E1008091E2008F7E8093E2008091E2
:1034F000E20081608093E20080914F04882311F004
:1035000084E007C08091E30087FD02C081E001C034
:1035100083E0809353040E9477168091E10083FF3B
:1035200029C08091E20083FF25C08091E100877F60
:103530008093E10082E08093530410924F048091C5
:10354000E1008E7F8093E1008091E2008E7F809386
:10355000E2008091E20080618093E20042E060E05E
:1035600080E00E94F8188091F00088608093F0005D
:103570000E947516FF91EF91BF91AF919F918F912E
:103580007F916F915F914F913F912F910F900FBE5F
:103590000F901F9018951F920F920FB60F92112443
:1035A0002F933F934F935F936F937F938F939F934B
:1035B000AF93BF93CF93DF93EF93FF93C091E90055
:1035C000CF708091EC00D82FD17080FDD0E81092A0
:1035D000E9008091F000877F8093F00078940E944A
:1035E0000F1B1092E9008091F00088608093F0003A
:1035F000CD2BCF70C093E900FF91EF91DF91CF9178
:10360000BF91AF919F918F917F916F915F914F91FA
:103610003F912F910F900FBE0F901F9018951F9301
:10362000CF93DF93CDB7DEB7AA970FB6F894DEBF7E
:103630000FBECDBFE4E5F4E088E08E0F9091F1007D
:1036400091938E13FBCF0E948D168091E80083FF2B
:103650001FC18091540490915504492F50E04A3085
:10366000510508F015C1FA01EC59FF4F0C942132B5
:10367000803881F0823809F00BC1809158048F7036
:103680008093E9008091EB0085FB882780F91092F8
:10369000E90006C08091500490915104911182601C
:1036A0009091E800977F9093E8008093F10010924A
:1036B000F100C8C0282F2D7F09F0EAC0882319F037
:1036C000823061F0E5C080915604813009F0E0C09D
:1036D000933009F080E0809351042BC08091560410
:1036E000811127C0809158048F7009F4D1C0809354
:1036F000E9002091EB0020FF1CC0933021F4809161
:10370000EB00806214C09091EB0090619093EB000D
:1037100021E030E0A90102C0440F551F8A95E2F76D
:103720004093EA001092EA008091EB008860809359
:10373000EB001092E9008091E800877F86C081113C
:10374000A7C0109156041F778091E3008078812BE9
:103750008093E3008091E800877F8093E8000E94D7
:103760002D198091E80080FFFCCF8091E3008068F4
:103770008093E300111102C082E001C083E08093D6
:10378000530486C08058823008F082C0809156046D
:10379000909157048C3D53E0950779F583E08A8337
:1037A0008AE289834FB7F894DE01139620E03EE069
:1037B00051E2E32FF0E050935700E49120FF03C063
:1037C000E295EF703F5FEF708E2F90E0EA3010F0DF
:1037D000C79601C0C0968D939D932F5F243149F702
:1037E0004FBF8091E800877F8093E8006AE270E035
:1037F000CE0101960E94341814C0AE014F5F5F4F96
:10380000609158040E947B17BC01009709F440C0E6
:103810009091E800977F9093E80089819A810E94B7
:1038200097188091E8008B778093E80031C080384A
:1038300079F58091E800877F8093E80080914F04BC
:103840008093F1008091E8008E778093E8000E94D9
:103850002D191EC081111CC0909156049230C0F4E5
:103860008091E800877F8093E80090934F040E9446
:103870002D1980914F04811106C08091E30087FDCE
:1038800002C081E001C084E0809353040E94791655
:103890008091E80083FF0AC08091E800877F8093D1
:1038A000E8008091EB0080628093EB00AA960FB64F
:1038B000F894DEBF0FBECDBFDF91CF911F91089569
:1038C0000895CF93809153048823A1F0C091E9001B
:1038D000CF709091EC00892F817090FD80E8C82B0B
:1038E0001092E9008091E80083FD0E940F1BCF70C9
:1038F000C093E900CF9108959093D3038093D203AE
:103900000895E091D203F091D303309721F0019014
:10391000F081E02D099480E00895E091D203F091C8
:10392000D303309721F00280F381E02D09940895AC
:10393000E091D203F091D303309721F00480F58118
:10394000E02D099408952091D0033091D10382177E
:10395000930771F09093D1038093D003E091D20349
:10396000F091D303309721F00680F781E02D099480
:1039700008952091CE033091CF038217930771F001
:103980009093CF038093CE03E091D203F091D303C1
:10399000309721F00084F185E02D09940895089571
:1039A0000C94CF1C0E9456280E94140E0E94DC2802
:1039B0000C94902D5F926F927F928F929F92AF9214
:1039C000BF92CF92DF92EF92FF920F931F93CF930C
:1039D000DF9300D000D01F92CDB7DEB70E94590E02
:1039E0009DEDC92E93E0D92E03E010E0AA24A39404
:1039F000B12C502E802F0E94D40E4C01F6017290F3
:103A000062906F016826792661147104A1F4015057
:103A1000110978F78FEF89838A831B820E945F28C0
:103A20008160782F9D838C8349815A816B818D8140
:103A30000E948A1D38C08091320481FD0E94DD0EF3
:103A40002BE030E07501022E02C0EE0CFF1C0A9440
:103A5000E2F7C70186219721892B09F129835A8230
:103A60008E209F2091E0892809F490E09B830E949A
:103A70005F288160782F9D838C8349815A816B8177
:103A80008D810E948A1D000F111FF801EB52FC4F1F
:103A900080819181E826F926F182E08204C02150DC
:103AA000310980F6B4CF0E94C82A1091D4030E9435
:103AB000811C1817D1F00E94811C8093D4030F90B1
:103AC0000F900F900F900F90DF91CF911F910F915A
:103AD000FF90EF90DF90CF90BF90AF909F908F902E
:103AE0007F906F905F900C94FE0D0F900F900F9051
:103AF0000F900F90DF91CF911F910F91FF90EF905A
:103B0000DF90CF90BF90AF909F908F907F906F90FD
:103B10005F900895CF93DF93CDB7DEB72B970FB6A5
:103B2000F894DEBF0FBECDBF4F83588769877A8771
:103B30008B87DE01119686E0FD0111928A95E9F7E7
:103B400085E0FE01379601900D928A95E1F7498153
:103B50005A816B817C818D819E810E9401242B96EC
:103B60000FB6F894DEBF0FBECDBFDF91CF910895A1
:103B7000CF93882309F4C2C0C82F823859F40E9419
:103B8000811C81FDBBC089E30E94DB260E94A8271F
:103B900089E30CC0833879F40E94811C80FDAEC09B
:103BA00083E50E94DB260E94A82783E50E941D274B
:103BB000CF910C94A827843859F40E94811C82FD6F
:103BC0009DC087E40E94DB260E94A82787E4EECFF1
:103BD0008CEF8C0F813A48F48C2F0E94F82C8111C5
:103BE0008DC08C2F0E94DB26E3CF80E28C0F8830C3
:103BF00048F4C77081E001C0880FCA95EAF70E94B7
:103C00006127D6CF8BE58C0F833078F4C53A29F045
:103C1000C63A31F083E890E005C081E890E002C048
:103C200082E890E0CF910C94A31C88E58C0F83313F
:103C300008F064C0C83A39F1C93A41F1CA3A49F1C9
:103C4000CB3A51F1CC3A59F1CD3A61F1C03B69F12F
:103C5000CE3A71F1CF3A79F1C13B81F1C23B89F1A2
:103C6000C33B91F1C43B99F1C53BA1F1C63BA9F11E
:103C7000C73BB1F1C83BB9F1C93BC1F1CA3BC9F17E
:103C800080E090E038C082EE90E035C089EE90E0B0
:103C900032C08AEE90E02FC085EB90E02CC086EB1E
:103CA00090E029C087EB90E026C08CEC90E023C028
:103CB0008DEC90E020C083E891E01DC08AE891E09F
:103CC0001AC082E991E017C084E991E014C081E252
:103CD00092E011C083E292E00EC084E292E00BC059
:103CE00085E292E008C086E292E005C087E292E0B9
:103CF00002C08AE292E0CF910C94B91CCF91089552
:103D0000882309F44BC0823859F40E94811C81FF3A
:103D100045C089E30E94DB260E94A82789E30CC0E6
:103D2000833871F40E94811C80FF38C083E50E94B3
:103D3000DB260E94A82783E50E941D270C94A82754
:103D4000843859F40E94811C82FF28C087E40E94B5
:103D5000DB260E94A82787E4EFCF9CEF980F913ACB
:103D600058F390E2980F983050F4877091E001C0BA
:103D7000990F8A95EAF7892F0E946727DFCF9BE585
:103D8000980F933020F480E090E00C94A31C885AA4
:103D9000833120F480E090E00C94B91C08958823CE
:103DA00021F00E9461270C94A8270895882321F010
:103DB0000E9467270C94A82708957F928F929F9264
:103DC000AF92BF92CF92DF92EF92FF920F931F9329
:103DD000CF93DF931F92CDB7DEB77C01C62E772E2F
:103DE000FC01058102950F70128111110E947E273E
:103DF0000E94D426882379F0112369F080E28C0D8B
:103E0000883048F082E00E94BD260E94D42691E0CE
:103E1000D82ED92601C0D12CE72DE295EF70F0E025
:103E2000E259FF4F0C942132872D807F072D0F70B0
:103E3000882311F00295007F112389F0002309F4F3
:103E400099C180E28C0D883020F4802F0E94612778
:103E500003C0802F0E9471270E94A8278BC18C2D40
:103E60000E94801E002309F4C3C180E28C0D8830BB
:103E700020F4802F0E94672703C0802F0E9477279D
:103E80000E94A827B5C1872D807F972D9F70803213
:103E900011F4892F03C0892F8295807FCC2021F0D7
:103EA000F1E0CF16A1F01DC0112339F0002319F164
:103EB000013009F50E9491279BC1002319F00130C0
:103EC00009F496C189830E949427898110C1112326
:103ED00021F0063008F08CC10EC0053008F088C112
:103EE00006C1112359F0002331F0F701958190FFAD
:103EF00041C19F7095830E94CF1E7AC1002309F4AF
:103F0000F6C03EC1872D86958695837090E0009718
:103F100019F0019761F06CC1112321F08C2D972DC0
:103F2000937002C080E090E00E94A31C61C1112345
:103F300021F08C2D972D937002C080E090E00E94BC
:103F4000B91C56C18C2D112319F00E94D02902C032
:103F50000E94382A0E94BD2A4BC1872D837009F028
:103F600052C0111145C18C2D829586958770880F9E
:103F7000880F9C2D9F70892E912CA12CB12C082E7E
:103F800004C0880C991CAA1CBB1C0A94D2F7C4FE5E
:103F900014C00FE010E020E030E0B901A80104C037
:103FA000440F551F661F771F8A95D2F7CB01BA01C0
:103FB000609570958095909503C060E070E0CB01AE
:103FC000272D26952695237030E02230310569F0A3
:103FD0002330310589F0682979298A299B292130E4
:103FE000310571F00E94492503C1682979298A2980
:103FF0009B290E946525FCC00E944925C501B4018A
:104000000E942D25F5C0112319F0872D817001C064
:104010008695882309F4ECC08C2D8295869587704F
:10402000880F880F9C2D9F70892E912CA12CB12C6C
:10403000082E04C0880C991CAA1CBB1C0A94D2F739
:10404000C4FE14C00FE010E020E030E0B901A80188
:1040500004C0440F551F661F771F8A95D2F7CB0106
:10406000BA01609570958095909503C060E070E00E
:10407000CB01272D269526952370422F50E0423004
:10408000510569F04330510589F0682979298A2959
:104090009B294130510571F00E942326A9C068294F
:1040A00079298A299B290E943F26A2C00E942326A3
:1040B000C501B4010E9407269BC08C2D90E0FC0135
:1040C000E05EF109E531F10508F050C0E258FF4F1C
:1040D0000C9421320C2D0F70872D8F71112321F03C
:1040E0000E94A025802F07CF0E94C125802F0E940B
:1040F000D61E7EC0112341F0053008F079C0872D0F
:104100008F710E94E62574C0063008F071C0F7CFA9
:10411000112339F0872D8F710E94A02569C01123CA
:10412000C9F3872D8F710E94C12562C0112329F028
:10413000872D8F710E948B255BC00E94812558C0FE
:10414000112351F0172D1F71812F0E94A02563E0CC
:10415000812F0E94B4264CC081E00E94BD2602300F
:1041600008F446C082E00E94BD2642C0112331F00F
:10417000002381F28C2D0E94B81D3AC0002389F2E1
:104180008C2D0E94801E34C0472D4F706C2DC701AE
:104190000E94E0060E94A5242BC0111129C0472DC2
:1041A0004F7050E042305105B9F04CF441155105C3
:1041B00081F041305105E1F40E94B82D19C043301F
:1041C000510569F04430510599F48C2D0E940A2E56
:1041D0000FC00E94A12D0CC00E94D42D09C00E94C6
:1041E000E72D06C0472D4F706C2DC7010E949F0A16
:1041F000DD20F9F00E94B02680FD1BC0F70112827D
:104200000E94AA260E94A025C7010E9428210E9480
:10421000AA260F90DF91CF911F910F91FF90EF9001
:10422000DF90CF90BF90AF909F908F907F900C9435
:10423000C1250F90DF91CF911F910F91FF90EF90CB
:10424000DF90CF90BF90AF909F908F907F90089518
:104250000F931F93CF93DF93EC01888199812B817A
:104260003C81232BB9F09F3F11F48F3F99F0CE0191
:104270000E949E08882371F0688179818A810E945A
:10428000A6268C010E945B260E942225B801CE0141
:104290000E94DD1EDF91CF911F910F9108950E9422
:1042A0007E270E948E270E9453270E94A8270E94E3
:1042B0006E2B0E94BD2A80E090E00E94A31C80E04B
:1042C00090E00C94B91C0E946E270C944F210E9420
:1042D0009B26292F22952F7030E02C3031054CF48D
:1042E0002A3031056CF42250310922303105A8F40E
:1042F00007C02C30310569F02F30310551F00DC069
:10430000803F69F018F4803E40F409C0843F29F4EE
:1043100006C093FB882780F9089580E0089581E026
:104320000895CF93DF9300D000D01F92CDB7DEB7B2
:104330000F900F900F900F900F90DF91CF910895F5
:10434000CF93DF9300D000D000D0CDB7DEB7269654
:104350000FB6F894DEBF0FBECDBFDF91CF910895A9
:104360001F93CF93DF93C091DD0316E08091DE03AE
:10437000C81799F0D0E01C9FF0011D9FF00D11248B
:10438000E152FC4F4081518162817381848195812A
:104390000E94A0212196C770E9CFDF91CF911F9194
:1043A000089540910F045091100460911104709190
:1043B000120480911304909114040C94A021809114
:1043C000140482958F7009F054C0809111048823E1
:1043D00009F44FC08091DD03A091DE0360910F04CA
:1043E000709110044091120450911304B6E08A17A2
:1043F00009F43FC090E041155105C1F17F3F11F430
:104400006F3FA1F1B89FF001B99FF00D1124E15267
:10441000FC4F218172132AC02081621327C02281A0
:10442000211124C0238134812417350710F4215031
:104430003109241B350B283C3105C0F420911404AC
:104440002F7020612093140426E0289FF001299FFB
:10445000F00D1124EC51FC4F80818F7080618083BE
:104460008FE094E00E9428210C94B021019687707F
:10447000BECF0895CF92DF92EF92FF920F931F93DA
:10448000CF93DF93CDB7DEB762970FB6F894DEBF58
:104490000FBECDBF8C0185E0F801DE011D960190B5
:1044A0000D928A95E1F7D8014C9111965C91119784
:1044B00012966C9112971396CD90DC9014973091D0
:1044C0000F047091100480911204909113040097CE
:1044D00009F46BC17F3F19F43F3F09F466C1E090D6
:1044E0001104EE2009F4C0C020911404C816D906A6
:1044F00028F0F601E81BF90BCF0104C080959095D8
:104500008C0D9D1DFF24F394883C910578F0F12CCF
:10451000207F09F0C6C07C2DD98AC88A89890E946B
:1045200091218FE094E00E942821B1C0822F807FEA
:1045300009F046C0751314C0341312C0611110C0C5
:104540002F702061209314040E94D1218FE094E009
:104550000E94282180911404D80115968C932EC0B6
:10456000CD2819F15F3F11F44F3FF9F0F62E61119C
:104570001CC08091DD032091DE0336E0821709F430
:104580005AC090E0389FF001399FF00D1124E1529C
:10459000FC4F7181571306C07081471303C07281AD
:1045A000711103C001968770E9CFF62E662309F4D6
:1045B00018C180911404816080931404F12C11C1FE
:1045C000751308C0341306C0611104C0809114042F
:1045D000D801C3C04D875E878D859E856A8B0E94FA
:1045E00067216A898823E1F16623D1F120911404BF
:1045F000822F82958F7090E0029774F080910F0463
:104600009091100498878F831986DB86CA862C8741
:10461000CE0107960E94282186E0F801AFE0B4E0C1
:1046200001900D928A95E1F70E94DF210E94D1212D
:10463000FF24F394D6C04D875E878D859E850E94AA
:104640009B26292F22952F7030E0223031050CF067
:10465000BCC09F7009F0B6C0805E883008F4C1C04D
:10466000C8010E942821E4CFC816D90608F453C017
:10467000F601E81BF90BCF01883C910508F450C006
:10468000F12C7C2DD98AC88A89890E949121EFE07A
:10469000F4E086E0DF011D928A95E9F70E94D121BE
:1046A000A0C0751314C0341312C0611110C08091E2
:1046B0001404F8018583C8010E94282186E0EFE0F8
:1046C000F4E0DF011D928A95E9F7FE2C8AC04D8740
:1046D0005E878D859E856A8B0E9467216A89882303
:1046E00009F4BECF662309F4BBCF20911404822FB6
:1046F00082958F7090E002970CF48ECF80910F041A
:10470000909110049A8389831B82DD82CC822E8350
:10471000CE0101967FCF809590958C0D9D1DACCFDD
:10472000F62E662309F49CCF75132EC034132CC0CB
:104730002091140420FD1FC0822F82958F70D9F024
:10474000D80115962C9315978F3049F08F5F982FCD
:104750009295907F822F8F70892B15968C93C8012C
:104760000E94282186E0F801AFE0B4E001900D92AC
:104770008A95E1F793CF86E0F801AFE0B4E00190CD
:104780000D928A95E1F72DC04D875E878D859E85B8
:104790000E946721811140CF809114048160809331
:1047A0001404C8010E9428211CC0662309F458CFB4
:1047B0004D875E878D859E850E946721882309F439
:1047C0004FCF2ACF811148CF0CC0243031050CF0D7
:1047D00047CF9F7009F440CFF8019581907F09F091
:1047E0003BCF8F2D62960FB6F894DEBF0FBECDBFC4
:1047F000DF91CF911F910F91FF90EF90DF90CF90BD
:1048000008951F93CF93DF93CDB7DEB72C970FB6E4
:10481000F894DEBF0FBECDBF4F83588769877A8774
:104820008B879C87CE0107960E943A22882369F0E5
:104830008F8198852A853B85232BF1F19F3F09F0D5
:1048400063C08F3F09F060C037C086E0FE01379635
:10485000DE01119601900D928A95E1F76F817885BE
:10486000EA85FB85309741F17F3F11F46F3F21F1DD
:104870002091DE0330E0C9010196877099274091AD
:10488000DD0350E08417950709F447C069837A83F4
:10489000FD83EC8396E0929FD001939FB00D11248D
:1048A000A152BC4FFE01319601900D929A95E1F70D
:1048B0008093DE030E94B02116E08091DD03909189
:1048C000DE038917C1F1189FC001112481529C4F4A
:1048D0000E943A22882379F1E091DD031E9FF001C6
:1048E0001124E152FC4F40815181628173818481A6
:1048F00095810E94A0218091DD0390E00196877050
:1049000099278093DD03D9CF4F81588569857A85B2
:104910008B859C850E94A021CFCF0E94632110929D
:10492000DE031092DD03EFE0F4E086E0DF011D928C
:104930008A95E9F7C1CF2C960FB6F894DEBF0FBE6B
:10494000CDBFDF91CF911F910895EF92FF920F930A
:104950001F93CF93DF938C01009709F46CC0F12C67
:10496000EE24E394E8012196F8018491843740F421
:10497000843008F051C0813081F0823019F15BC081
:10498000853709F444C0A8F19CE7980F903708F0E8
:1049900052C08F770E94801E41C00E5F1F4FFE01E4
:1049A000C49180E28C0F883048F4C7708E2D01C00E
:1049B000880FCA95EAF70E94812714C08C2F0E94A5
:1049C000B81D2DC00E5F1F4FFE01C49180E28C0FF9
:1049D000883058F4C7708E2D01C0880FCA95EAF749
:1049E0000E9487270E94A8271AC08C2F0E94801E31
:1049F00016C00E5F1F4FFE01C491CC2381F08FE9DA
:104A00009FE00197F1F700C00000C150F6CF0E5FA4
:104A10001F4FFE01F49003C00E94B81D8E018F2D20
:104A2000882309F49FCFEFE9FFE03197F1F700C049
:104A300000008150F5CFDF91CF911F910F91FF9032
:104A4000EF90089508956093190470931A04809369
:104A50001B0490931C040C944F210F931F930091FF
:104A6000190410911A0420911B0430911C04DC01DC
:104A7000CB01802B912BA22BB32B80931904909305
:104A80001A04A0931B04B0931C041F910F910C9463
:104A90004F210F931F930091190410911A04209134
:104AA0001B0430911C04DC01CB0180239123A22341
:104AB000B3238093190490931A04A0931B04B0931A
:104AC0001C041F910F910C944F210F931F93009181
:104AD000190410911A0420911B0430911C04DC016C
:104AE000CB0180279127A227B327809319049093A5
:104AF0001A04A0931B04B0931C041F910F910C94F3
:104B00004F2110921504109216041092170410925F
:104B100018040C944F2141E050E060E070E004C0C4
:104B2000440F551F661F771F8A95D2F740931504CF
:104B30005093160460931704709318040C944F213B
:104B400041E050E060E070E004C0440F551F661F74
:104B5000771F8A95D2F78091150490911604A09141
:104B60001704B0911804482B592B6A2B7B2B4093C8
:104B700015045093160460931704709318040C9452
:104B80004F2141E050E060E070E004C0440F551F49
:104B9000661F771F8A95D2F740955095609570955E
:104BA0008091150490911604A0911704B0911804F7
:104BB000482359236A237B234093150450931604FA
:104BC00060931704709318040C944F2141E050E057
:104BD00060E070E004C0440F551F661F771F8A9580
:104BE000D2F78091150490911604A0911704B0910A
:104BF0001804482759276A277B27409315045093A8
:104C0000160460931704709318040C944F210F93AB
:104C10001F930091150410911604209117043091F0
:104C20001804DC01CB01802B912BA22BB32B80939A
:104C3000150490931604A0931704B09318041F91C1
:104C40000F910C944F210F931F9300911504109115
:104C500016042091170430911804DC01CB01802345
:104C60009123A223B3238093150490931604A09359
:104C70001704B09318041F910F910C944F210F93B8
:104C80001F93009115041091160420911704309180
:104C90001804DC01CB0180279127A227B32780933A
:104CA000150490931604A0931704B09318041F9151
:104CB0000F910C944F210895CF92DF92EF92FF92C3
:104CC0000F931F93CF93DF938C01C0901904D09062
:104CD0001A04E0901B04F0901C048091150490913C
:104CE0001604A0911704B0911804C82AD92AEA2AF8
:104CF000FB2ACFE1D0E0D701C6010C2E04C0B69547
:104D0000A795979587950A94D2F780FF06C0B801BA
:104D10008C2F0E94240D019721F4219760F780E0E9
:104D200001C08C2FDF91CF911F910F91FF90EF90D9
:104D3000DF90CF900895CF93DF93EC010E945C2623
:104D4000BE010E94240DDF91CF910895CB010E94F6
:104D50009B26089580911D048595859585950895D8
:104D600080911D048770089598E0899F9001112417
:104D7000262B20931D040C94A02520911D048095C2
:104D8000822380931D04982F977069F430E0482F98
:104D9000552747FD50952417350729F085958595AA
:104DA00085950C94C125089590911D04977081E01C
:104DB00009F480E0089590912D02992321F09091BB
:104DC0002E02911109C020912F0230913002F90179
:104DD00032969FEF40E01FC0982F96959695969536
:104DE0009F3050F5E0912F02F0913002E90FF11D54
:104DF000877021E030E0A90102C0440F551F8A9559
:104E0000E2F7CA019181892B818308959F3F39F090
:104E10004F5F4E3041F051915813F8CF0DC05111F2
:104E2000F7CF942FF5CF9F3F39F0F901E90FF11D2E
:104E300097FDFA9582830895089590912D02992304
:104E400021F090912E02911109C020912F023091F2
:104E50003002F9013296205F3F4F1FC0982F969580
:104E6000969596959F30F0F4E0912F02F0913002E4
:104E7000E90FF11D877021E030E0A90102C0440F65
:104E8000551F8A95E2F7CA01809591818923818314
:104E900008953196E217F30729F090819813F9CF1E
:104EA0001082F7CF089581E090E0E0912F02F09119
:104EB0003002E80FF91F1082019680319105A9F7A1
:104EC000089590913104892B809331040895809541
:104ED0009091310489238093310408951092310414
:104EE000089590913004892B809330040895809523
:104EF00090913004892380933004089510923004F7
:104F0000089590912F04892B80932F040895809504
:104F100090912F04892380932F04089510922F04D9
:104F2000089580931E04089510921E0408958091A0
:104F30002F0290913002FC0131969C01205F3F4F7F
:104F400080E0919191118F5FE217F307D1F70895F7
:104F5000E0912F02F0913002809131048083E09142
:104F60002F02F0913002908180913004892B808350
:104F7000E0912F02F0913002908180912F04892BD3
:104F8000808380911E04882361F0E0912F02F091CC
:104F900030029081892B80830E9497278111109283
:104FA0001E0480912F02909130020C948D1C20E001
:104FB000009739F0AC0141505109842395232F5FAC
:104FC000F7CF822F089580915304843039F11092E5
:104FD000330420E488E190E00FB6F894A89580931C
:104FE00060000FBE2093600080E00E940E0680E00B
:104FF0000E94FE0D83B7817F846083BF83B7816089
:1050000083BF7894889583B78E7F83BF88E10FB67E
:10501000F89480936000109260000FBE0895089588
:10502000089580E00E940E060E940F280E94590EEB
:105030000E9410280E94DE0E91E0811101C090E0D4
:10504000892F08950E94632180E00E940E060E942D
:10505000902D0E94811C0C94FE0D1F920F920FB692
:105060000F9211248F939F93AF93BF93809133043A
:10507000811113C08091340490913504A0913604BD
:10508000B09137044196A11DB11D809334049093D3
:105090003504A0933604B0933704BF91AF919F912C
:1050A0008F910F900FBE0F901F90189582E084BDD6
:1050B00093E095BD9AEF97BD80936E0008952FB74A
:1050C000F8948091340490913504A0913604B09105
:1050D00037042FBF0895CF92DF92EF92FF920F9384
:1050E0001F932FB7F8944091340450913504609188
:1050F0003604709137042FBF6A017B01EE24FF2430
:105100008C0120E030E0C016D106E206F30610F470
:10511000415051099A01281B390BC9011F910F9168
:10512000FF90EF90DF90CF9008951F920F920FB6EF
:105130000F9211248F939F93AF93BF938091340468
:1051400090913504A0913604B09137040196A11DC9
:10515000B11D8093340490933504A0933604B0932A
:105160003704BF91AF919F918F910F900FBE0F9019
:105170001F9018950E947E19F8942FEF87EA91E608
:10518000215080409040E1F700C0000087E090EBA4
:10519000DC0180935E0490935F04A0936004B0935D
:1051A00061049CE088E10FB6F894A89580936000B4
:1051B0000FBE90936000FFCF0E941B29811102C097
:1051C0000E94F7280E942629809332040E943329E6
:1051D00080935C0487FB882780F980932E020E94CD
:1051E0002A29682F70E080E090E00C9423256DEE72
:1051F0007EEF80E090E00E94473260E082E090E045
:105200000E94353260E083E090E00E94353260E039
:1052100084E090E00E94353260E085E090E00E94FA
:10522000353260E086E090E00E9435326FEF87E033
:1052300090E00C94353280E090E00E942F3221E023
:105240008D3E9E4F09F020E0822F089582E090E08D
:105250000C94273283E090E00C942732682F83E08F
:1052600090E00C94353284E090E00C942732682F63
:1052700084E090E00C94353286E090E00C94273284
:10528000682F86E090E00C94353287E090E00C9433
:105290002732682F87E090E00C94353280913A04F1
:1052A00080FF0BC06091340285E0689FB00111243B
:1052B00075956795759567952BC081FF09C06091BD
:1052C000340285E0689FB00111247595679520C070
:1052D00082FF07C06091340285E0689FB00111240D
:1052E00017C090913B049923D1F060913302961737
:1052F00088F72091340285E0289F90011124929F25
:10530000A001939F500D112470E0CA010E940D323C
:105310006038710540F46115710539F002C065E02F
:1053200070E0862F08958FE7089581E008958091B9
:105330003A0480FF08C06091320270E0759567956D
:105340007595679521C081FF06C06091320270E0BB
:105350007595679519C082FF04C06091320270E0B4
:1053600010C090913B049923C1F0609131029617CF
:10537000A0F780913202899FC001112470E00E9441
:105380000D326038710528F46115710521F0862F02
:1053900008958FE7089581E0089561E070E0F4CF0B
:1053A000803F21F40E944E29819504C0813F29F459
:1053B0000E944E2980933E040895823F21F40E946A
:1053C0004E29819504C0833F29F40E944E29809381
:1053D0003D040895893F19F40E94972905C08A3F2A
:1053E00031F40E949729819580933F0408958B3F63
:1053F00021F40E949729819504C08C3F29F40E94D2
:105400009729809340040895843F21F480913C04BF
:10541000816017C0853F21F480913C04826011C0F7
:10542000863F21F480913C0484600BC0873F21F4C7
:1054300080913C04886005C0883F31F480913C0431
:10544000806180933C0408958D3F21F480913A045B
:1054500081600BC08E3F21F480913A04826005C0C8
:105460008F3F29F480913A04846080933A04089530
:10547000803F39F480913E0487FF6CC010923E0457
:1054800069C0813F29F480913E041816BCF362C0C4
:1054900090913D04823F29F497FF5CC010923D0437
:1054A00059C0833F19F41916CCF354C0893F41F415
:1054B00080913F0418160CF04DC010923F044AC072
:1054C0008A3F29F480913F0487FF44C0F6CF8B3F89
:1054D00039F48091400487FF3DC0109240043AC0E7
:1054E0008C3F29F4809140041816BCF333C0843FEC
:1054F00021F480913C048E7F17C0853F21F4809178
:105500003C048D7F11C0863F21F480913C048B7F49
:105510000BC0873F21F480913C04877F05C0883F02
:1055200031F480913C048F7E80933C0413C08D3F06
:1055300021F480913A048E7F0BC08E3F21F480913C
:105540003A048D7F05C08F3F29F480913A048B7F08
:1055500080933A0480913D0481110EC080913E04F5
:1055600081110AC080913F04811106C080914004DE
:10557000811102C010923B0408958CE394E00E94D4
:10558000981C0E945F2890933904809338040895F2
:105590001F93CF93DF9380913804909139040E9438
:1055A0006B28AC0190913B04992321F020913502A6
:1055B00030E006C0209136028AE0289F9001112435
:1055C0004217530708F486C080913D04C0913E0401
:1055D000D0913F0410914004811107C0C11176C0E1
:1055E000D11174C0111172C075C09F3F19F09F5F37
:1055F00090933B04181624F40E944E2980933D0496
:1056000080913D0487FF05C00E944E2981958093BB
:105610003D041C1624F40E944E2980933E04809180
:105620003E0487FF05C00E944E29819580933E0469
:1056300060913D04662339F1C0913E04CC2319F1F9
:10564000772767FD7095872F972F0E942F2F23E3D1
:1056500033E343E35FE30E943F300E94FC2E6093FC
:105660003D046C2F772767FD7095872F972F0E9439
:105670002F2F23E333E343E35FE30E943F300E9495
:10568000FC2E60933E041D1624F40E9497298093FB
:105690003F0480913F0487FF05C00E9497298195B0
:1056A00080933F04111624F40E94972980934004AC
:1056B0008091400487FF05C00E94972981958093BF
:1056C0004004DF91CF911F910C94BD2A9F3F09F0B8
:1056D0008ECF96CFDF91CF911F910895ECE3F4E048
:1056E00085E0DF011D928A95E9F710923B04109244
:1056F0003A040895833081F128F4813059F08230E2
:10570000D1F00895853009F449C0B8F1863009F424
:1057100056C0089580913602262F30E0280F311DA3
:105720002F3F310524F4680F6093360208958FEF00
:1057300080933602089580913502262F30E0280F9D
:10574000311D2F3F310524F4680F60933502089511
:105750008FEF80933502089580913402262F30E038
:10576000280F311D2F3F310524F4680F6093340258
:1057700008958FEF80933402089580913302262F8D
:1057800030E0280F311D2F3F310524F4680F60935E
:10579000330208958FEF809333020895809132028F
:1057A000262F30E0280F311D2F3F310524F4680FDC
:1057B0006093320208958FEF8093320208958091B2
:1057C0003102262F30E0280F311D2F3F310524F400
:1057D000680F6093310208958FEF8093310208952E
:1057E000833011F128F4813049F0823091F008952E
:1057F000853081F120F18630C1F108958091360223
:10580000681720F4861B80933602089510923602A2
:10581000089580913502681720F4861B8093350225
:10582000089510923502089580913402681720F48B
:10583000861B80933402089510923402089580915B
:105840003302681720F4861B809333020895109268
:105850003302089580913202681720F4861B8093EA
:105860003202089510923202089580913102681731
:1058700020F4861B8093310208951092310208951E
:105880000F931F93873208F048C08E3108F08DC007
:10589000803109F477C008F5873009F461C068F4F5
:1058A000863009F09DC080913204817F8E7F809385
:1058B000320481E08093420494C08B3009F489C0A3
:1058C0008E3009F08DC08091320482FB222720F9AE
:1058D00091E0922790FB82F95EC0863109F479C08D
:1058E00060F4813109F07CC00E94632190912E0206
:1058F00081E0892780932E026CC0893109F469C048
:105900008B3109F06DC08091320481FB222720F990
:1059100091E0922790FB81F93EC0883309F459C089
:1059200050F4893209F457C0853309F454C08732E2
:1059300009F451C055C0833409F44DC028F48A33AA
:1059400008F44EC0895332C0883409F049C00E941F
:1059500063210E940E0F0E9495080E94BA2839C048
:1059600090913204892F8095817080FB90F929F005
:10597000966098609093320434C0997F977F90939B
:10598000320427C08091320483FB222720F991E062
:10599000922790FB83F9809332049923D1F0809170
:1059A000320481608093320414C08D5141E050E094
:1059B00060E070E08A019B0104C0000F111F221FEC
:1059C000331F8A95D2F7C901B8010E9423250E948E
:1059D000632181E006C061E070E080E090E0F5CFF7
:1059E00080E01F910F91089580E0089580E0089570
:1059F000CF93C82F80914204813069F018F0823033
:105A0000C9F184C0E0912F02F0913002808182328E
:105A100009F07EC007C0E0912F02F0913002808132
:105A2000823261F48C2F0E94F42C811104C08C2FDF
:105A30000E94402C1DC081E090E01AC08C2F0E9473
:105A4000F62C811114C0C43179F048F4CB3079F0D0
:105A5000C03109F061C082E08093420408C0C932BD
:105A600019F0C83321F058C01092420455C081E0AB
:105A7000817054C0C93291F120F5C43179F1B0F48C
:105A8000C73009F047C08EE18093360282E38093ED
:105A900035028AE08093340284E18093330288E007
:105AA0008093320288E28093310234C0CE51C630F6
:105AB00088F5EC2FF0E0EA50FD4F8081809341049F
:105AC00029C0CE34E9F020F4CB3421F56AE013C0CC
:105AD000C13579F0C235F1F461E00DC08091410427
:105AE000882319F01092410415C081E0809342048C
:105AF00015C061E006C0809141040E947A2B0AC063
:105B00006AE0809141040E94F02B04C0109242048C
:105B100080E004C081E002C080E0AACFCF91089568
:105B20000E941B29811102C00E94F7280E943C2973
:105B300080935D0480FF02C0869501C080E00C94D4
:105B40000E0680915D04982F9695292F30E0233022
:105B500031054CF49F5F990F8170892B8160809390
:105B60005D040E94402980915D0486950C940E0688
:105B700080915D04982F969591F09158990F8170BE
:105B8000892B80935D048E7F91E009F490E08091F1
:105B90005D0490FB80F980935D040E944029809110
:105BA0005D0486950C940E0680915D04982F909567
:105BB00090FB80F980935D040E94402980915D04F0
:105BC00080FF02C0869501C080E00C940E06909183
:105BD0005D04892F86958F5F8F779170843028F4CC
:105BE000880F892B80935D0402C090935D0480919F
:105BF0005D048E7F91E009F490E080915D0490FB5C
:105C000080F980935D040E94402980915D0486950F
:105C10000C940E0620915D04922F96958927982F5B
:105C2000990F822F8170892B80935D048E7F91E084
:105C300009F490E080915D0490FB80F980935D040D
:105C40000E94402980915D0486950C940E068091F7
:105C50005D04869508955058BB27AA270ED0D1C160
:105C6000C2D130F0C7D120F031F49F3F11F41EF4BF
:105C7000B7C10EF4E095E7FB9FC1E92FD3D180F3C4
:105C8000BA17620773078407950718F071F49EF539
:105C9000EBC10EF4E0950B2EBA2FA02D0B01B9012C
:105CA00090010C01CA01A0011124FF27591B99F092
:105CB000593F50F4503E68F11A16F040A22F232F9E
:105CC000342F4427585FF3CF469537952795A795EE
:105CD000F0405395C9F77EF41F16BA0B620B730B95
:105CE000840BBAF09150A1F0FF0FBB1F661F771F06
:105CF000881FC2F70EC0BA0F621F731F841F48F4BB
:105D0000879577956795B795F7959E3F08F0B3CF40
:105D10009395880F08F09927EE0F9795879508952A
:105D200027D108F481E008950CD06BC163D140F015
:105D30005AD130F021F45F3F19F03EC1511195C1A5
:105D40004FC170D198F39923C9F35523B1F3951B33
:105D5000550BBB27AA2762177307840738F09F5F8C
:105D60005F4F220F331F441FAA1FA9F333D00E2EFB
:105D70003AF0E0E830D091505040E695001CCAF768
:105D800029D0FE2F27D0660F771F881FBB1F26172D
:105D900037074807AB07B0E809F0BB0B802DBF0100
:105DA000FF2793585F4F2AF09E3F510568F004C1CA
:105DB0005CC15F3FECF3983EDCF386957795679581
:105DC000B795F7959F5FC9F7880F911D96958795B1
:105DD00097F90895E1E0660F771F881FBB1F6217D0
:105DE00073078407BA0720F0621B730B840BBA0B8E
:105DF000EE1F88F7E095089504D06894B11135C17D
:105E0000089518D188F09F5790F0B92F9927B7516E
:105E1000A0F0D1F0660F771F881F991F1AF0BA956E
:105E2000C9F712C0B13081F01FD1B1E008951CC193
:105E3000672F782F8827B85F39F0B93FCCF3869564
:105E400077956795B395D9F73EF4909580957095C1
:105E500061957F4F8F4F9F4F0895E89409C097FB3E
:105E60003EF490958095709561957F4F8F4F9F4F31
:105E70009923A9F0F92F96E9BB279395F695879575
:105E800077956795B795F111F8CFFAF4BB0F11F438
:105E900060FF1BC06F5F7F4F8F4F9F4F16C08823DF
:105EA00011F096E911C0772321F09EE8872F762F15
:105EB00005C0662371F096E8862F70E060E02AF056
:105EC0009A95660F771F881FDAF7880F9695879542
:105ED00097F9089588D018F011F08CD038F480C06C
:105EE000C4C0E92F9FD0B0F35523C9F3E7FB621775
:105EF000730784079507A8F199F3E92FFF278823F3
:105F00002AF03197660F771F881FDAF7952F5527EC
:105F1000442332F091505040220F331F441FD2F7D8
:105F2000BB27E91BF50B621B730B840BB109C1F294
:105F300022F4620F731F841FB11D31972AF0660F80
:105F4000771F881FBB1FEFCF915050405AF041F090
:105F5000882332F0660F771F881F91505040C1F799
:105F6000939530C08695779567959F5FD9F7F8CF61
:105F7000990F0008550FAA0BE0E8FEEF161617065A
:105F8000E807F907C0F012161306E407F50798F0C2
:105F9000621B730B840B950B39F40A2661F0232BDB
:105FA000242B252B21F408950A2609F4A140A69557
:105FB0008FEF811D811D089597F99F6780E870E03C
:105FC00060E008959F3F31F0915020F487957795D8
:105FD0006795B795880F911D9695879597F90895C0
:105FE0009FEF80EC089500240A94161617061806F1
:105FF0000906089500240A941216130614060506CD
:106000000895092E0394000C11F4882352F0BB0F5D
:1060100040F4BF2B11F460FF04C06F5F7F4F8F4FC0
:106020009F4F089557FD9058440F551F59F05F3FFB
:1060300071F04795880F97FB991F61F09F3F79F0AA
:1060400087950895121613061406551FF2CF46952C
:10605000F1DF08C0161617061806991FF1CF8695AE
:106060007105610508940895E894BB276627772792
:10607000CB0197F908957CDF08F48FEF08950BD0DA
:10608000C0CFB1DF28F0B6DF18F0952309F094CF28
:10609000A7CF1124EACFC6DFA0F3959FD1F3950FC8
:1060A00050E0551F629FF001729FBB27F00DB11D9C
:1060B000639FAA27F00DB11DAA1F649F6627B00D2C
:1060C000A11D661F829F2227B00DA11D621F739F15
:1060D000B00DA11D621F839FA00D611D221F749F23
:1060E0003327A00D611D231F849F600D211D822F6A
:1060F000762F6A2F11249F5750408AF0E1F08823B1
:106100004AF0EE0FFF1FBB1F661F771F881F9150BD
:106110005040A9F79E3F510570F04ECFA6CF5F3F8C
:10612000ECF3983EDCF3869577956795B795F795F0
:10613000E7959F5FC1F7FE2B880F911D9695879578
:1061400097F90895FA01EE0FFF1F309621053105EA
:1061500099F16115710561F48038BFE39B0749F13E
:1061600068949038810561F08038BFEF9B0741F05B
:10617000992342F5FF3FE1053105210511F1E8942E
:106180000894E795D901AA2329F4AB2FBE2FF85F15
:10619000D0F310C0FF5F70F4A695E0F7F73950F028
:1061A00019F0FF3A38F49F779F930CD00F9007FCBB
:1061B000905808953EF014CF60E070E080E89FE3CF
:1061C00008954FE79F775F934F933F932F939ED010
:1061D0002F913F914F915F9152DF05C019F40EF05E
:1061E000EBCE42CFFDCE26DFC8F39638C0F707F8D6
:1061F0000F92E8942BE33AEA48EB5FE74EDF0F9209
:106200000F920F924DB75EB70F92C0D0E6E2F1E069
:1062100016D04F915F91EF91FF91E595EE1FFF1F13
:1062200049F0FE57E0684427EE0F441FFA95E1F766
:106230004195550B32D00F9007FE26C00895DF938D
:10624000CF931F930F93FF92EF92DF927B018C010C
:10625000689405C0DA2EEF011EDFFE01E894A591D7
:106260002591359145915591AEF3EF0106DDFE0183
:106270009701A801DA9479F7DF90EF90FF900F91E2
:106280001F91CF91DF9108959B01AC0160E070E018
:1062900080E89FE349CD90CE95CECCDEE8F39923FC
:1062A000D9F3940F511DBBF39150504094F059F025
:1062B000882332F0660F771F881F91505040C1F736
:1062C0009E3F510544F7880F911D9695879597F944
:1062D00008955F3FACF0983E9CF0BB27869577957C
:1062E0006795B79508F4B1609395C1F7BB0F58F760
:1062F00011F460FFE8CF6F5F7F4F8F4F9F4FE3CF69
:10630000B4CE0EF05FCE6CCE689456CE93DEC8F35A
:106310009923D1F3C6F3DF93CF931F930F93FF928B
:10632000C92FDD2788232AF02197660F771F881F42
:10633000DAF720E030E040E85FEB9FE3883920F0B7
:10634000803E30F021968F7787DCEEE4F1E003C0E9
:1063500083DCEBE7F1E073DF8B01BE01EC01FB2E88
:106360006F5771097595771F880B990B78DD28E1B8
:1063700032E741E35FE38FDEAF2D9801AE01FF907E
:106380000F911F91CF91DF9178DC3BCEFA01DC01B8
:10639000AA0FBB1F9B01AC01BF5728F4222733274C
:1063A000442750781FC0B75188F4AB2F002446957E
:1063B00037952795011CA395D2F3002069F0220F91
:1063C000331F441FB395DAF30DD045CC613071050E
:1063D000A0E88A07B94630F49B01AC01662777270D
:1063E00088279078309621F020833183428353832D
:1063F0000895AA1BBB1B51E107C0AA1FBB1FA6170C
:10640000B70710F0A61BB70B881F991F5A95A9F75D
:1064100080959095BC01CD01089597FB072E16F449
:10642000009407D077FD09D00E94F93107FC05D010
:106430003EF4909581959F4F0895709561957F4F9B
:106440000895EE0FFF1F0590F491E02D0994F9993E
:10645000FECF92BD81BDF89A992780B50895A8E135
:10646000B0E042E050E00C944F32262FF999FECF75
:1064700092BD81BDF89A019700B4021639F01FBA97
:1064800020BD0FB6F894FA9AF99A0FBE08950196B6
:10649000272F0E9436320C943532DC01CB01FC01EF
:1064A000F999FECF06C0F2BDE1BDF89A319600B46D
:0E64B0000D9241505040B8F70895F894FFCF78
:1064BE000AA7CF44000000410000DC440000004168
:1064CE00000000000000804000005C4500004041DC
:1064DE00000000000000804052D0244500004041E2
:1064EE000AA7CF44000000410000DC440000004138
:1064FE00000000000000804052D0244500004041C2
:10650E00000000000000804000005C45000040419B
:10651E000AA7CF44000000410000DC440000004107
:10652E00000000000000804052D024450000404191
:10653E0000000000000080400AA74F4500004041C7
:10654E000AA7CF44000000410000DC4400000041D7
:10655E00000000000000804052D0244500000041A1
:10656E0000000000000080405CFF38450000004144
:10657E00000000000000804052D024450000004181
:10658E000AA7CF44000000410000DC440000004197
:10659E00000000000000804052D0244500008041E1
:1065AE0053D024450000404160970A450000004149
:1065BE0054D0A444000000410000DC44000000411F
:1065CE0060970A450000A041640007000CFF000020
:1065DE00003F6485151316F015BC15881501011FB3
:1065EE00042808140A321E0002040507090B0C0EBB
:1065FE001011131517181A1C1D1F212324262829C4
:10660E002B2D2F3032343537393B6966207965733F
:10661E000A097065616E7574206275747465720A0C
:10662E00656C73650A097269636520736E61636BCD
:10663E0073001F0F03764F5F6F7F496943790959C6
:10664E0053633149803F5D8B803FF8BF803FCAE185
:10665E00803F73ED803FCAE1803FF8BF803F5D8B86
:10666E00803F3149803F0000803FF16D7F3F75EAEA
:10667E007E3F4C827E3F833F7E3F84287E3F833F1A
:10668E007E3F4C827E3F75EA7E3FF16D7F3F00007C
:10669E00803F3F4D3639DF0A920A5C0A230AB6095B
:1066AE00CF09E809010A01020304050607080900DB
:00000001FF
